:100000000C942A001895000018950000189500001F
:10001000189500001895000018950000189500002C
:100020000C94A80118950000189500001895000080
:10003000189500001895000018950000189500000C
:1000400018950000189500001895000018950000FC
:10005000189500008FE58DBFC0EEE8E64E2E84E0D7
:100060008EBFD3E0F3E05F2EA89584B7082E877F7C
:1000700084BF88E1992781BD91BDEEEFF3E0A0E652
:10008000B0E088278D933197E9F78CE089B980E05B
:1000900080BD88E18AB9662480E08FBD84E08EBD92
:1000A0008EEE95E89DBD8CBD79B7746079BFB99A25
:1000B000C1980E94DF0484E690E00E940C058CE069
:1000C0000E94FD040E94C1040E94FE0570E071B907
:1000D00070E270B974E076BFB89A8F9A979880E012
:1000E00080938800E6EDF1E10E94A0040E94A7043D
:1000F000E6EDF1E10E94A0040E94A704E8EDF1E121
:100100000E94A0040E94A70479B7746079BF789414
:100110000E94C1040E94BD048FE711E00E94D00438
:10012000E6E0F2E10E94B6048FEB11E00E94D004F9
:10013000E8E1F2E10E94B604E3E0F0E00E94D604B8
:100140000E94C1040E94FC0100918800013011F05E
:100150000C94B800D201EAE2F2E10E945B0681E170
:100160000E9455060E94E701229681E10E945106F5
:100170000E94A80200918800013011F00C94CE007A
:10018000D201ECE3F2E10E945B0681E10E94550698
:100190000E94E701229681E10E9451068FE711E05B
:1001A0000E94D004EEE4F2E10E94B604EBE8F0E035
:1001B000A0E5B3E00E9422070E94AE048FEB11E09D
:1001C0000E94D004D201E9E8F0E00E943707D20192
:1001D0000E94B004E3E0F0E00E94D6040E94C10453
:1001E0008FE711E00E94D004E8E5F2E10E94B60436
:1001F0008FED0E94EF04E0E6F2E10E94B6048FEB7F
:1002000011E00E94D004EAE6F2E10E94B604ECE7B5
:10021000F2E10E94A0040E94A704E6EDF1E10E9431
:10022000A0040E94A704979AE6EDF1E10E94A004C1
:100230000E94A704E8E8F2E10E94A0040E94A7043B
:10024000E6EDF1E10E94A0040E94A7040E943003A1
:1002500000918800013011F00C943C01D201EEE9CC
:10026000F2E10E945B0682E10E9455060E94E701CE
:10027000229682E10E945106E3E9F0E00E947E07A7
:10028000E2ECF1E10E94D4080E94650718F011F039
:100290000C9468018FE71CE00E94D004A0E5B3E055
:1002A000AF93BF93E3E9F0E00E947E070E941B0535
:1002B00011E001E0BF91AF910E947206E0E5F3E02A
:1002C000A0E5B3E00E944C070E94AE040C948401A8
:1002D0008FE71DE00E94D004A0E5B3E0AF93BF9389
:1002E000E3E9F0E00E947E070E941B0511E001E0B7
:1002F000BF91AF910E947206E0E5F3E0A0E5B3E0A4
:100300000E944C070E94AE048FEB1DE00E94D004B7
:10031000A0E5B3E0AF93BF93E7E9F0E00E947E076A
:100320000E941B0511E001E0BF91AF910E9472068F
:10033000E0E5F3E0A0E5B3E00E944C070E94AE04C4
:10034000EEE1F0E00E94D6040C942601F894FFCF71
:100350000F921F922F923F924F925F927F92AF9295
:10036000BF920F931F932F933F934F935F936F937E
:100370007F938F939F93AF93BF93CF93DF93EF932D
:10038000FF938FB78F938EEE95E89DBD8CBD88B39C
:1003900091E0892788BB8F918FBFFF91EF91DF910B
:1003A000CF91BF91AF919F918F917F916F915F910D
:1003B0004F913F912F911F910F91BF90AF907F90E0
:1003C0005F904F903F902F901F900F9018950E9434
:1003D000C1048FE711E00E94D004E0EBF2E10E943B
:1003E000B6048FEB11E00E94D004A881B9810E946D
:1003F000B004F894FFCF0895E2ECF2E10E94A0046B
:100400000E94A70480E0809388000E94130662FA8D
:1004100016F00C940E0281E08093880018E80E9488
:10042000240662FA16F00C94180281E0809388008A
:1004300016E30E94240662FA16F00C94220281E070
:100440008093880012E80E94240662FA16F00C9449
:100450002C0281E08093880082E090E00E940C05ED
:100460000E94130662FA16F00C94390281E0809320
:10047000880019E80E94240662FA16F00C944302E0
:1004800081E0809388000E944106AEE8B0E01C93B2
:1004900062FA16F00C944F0281E0809388000E946B
:1004A0004106ADE8B0E01C9362FA16F00C945B02D2
:1004B00081E0809388000E944106A7E8B0E01C9389
:1004C00062FA16F00C94670281E0809388000E9423
:1004D0004106ACE8B0E01C9362FA16F00C9473028B
:1004E00081E0809388000E944106ABE8B0E01C9355
:1004F00062FA16F00C947F0281E0809388000E94DB
:100500004106A7E8B0E01C9362FA16F00C948B0247
:1005100081E0809388000E941E06E2EEF2E10E94D4
:10052000A004EBE8F0E0A0E5B3E00E9422070E94FF
:1005300098040E94A704E4EFF2E10E94A0040E9444
:10054000A704E6EDF1E10E94A0040E94A70408952B
:10055000E6E1F3E10E94A0040E94A70480E08093FA
:1005600088000E94130662FA16F00C94BA0281E029
:100570008093880018E80E94240662FA16F00C9412
:10058000C40281E08093880013EF0E94240662FA7F
:1005900016F00C94CE0281E0809388001DE20E9448
:1005A000240662FA16F00C94D80281E08093880049
:1005B00082E090E00E940C050E94130662FA16F099
:1005C0000C94E50281E08093880019E80E942406DB
:1005D00062FA16F00C94EF0281E0809388000E948A
:1005E0004106AAE8B0E01C9362FA16F00C94FB02F4
:1005F00081E0809388000E944106A9E8B0E01C9346
:1006000062FA16F00C94070381E0809388000E9440
:100610004106A7E8B0E01C9362FA16F00C941303AD
:1006200081E0809388000E941E06E4E3F3E10E94CB
:10063000A004D201E9E8F0E00E943707D2010E944D
:100640009A040E94A704E4E4F3E10E94A0040E943B
:10065000A704E6EDF1E10E94A0040E94A70408951A
:10066000E2E6F3E10E94A0040E94A70480E08093E8
:1006700088000E94130662FA16F00C94420381E08F
:100680008093880018E80E94240662FA16F00C9401
:100690004C0381E08093880014E20E94240662FAF1
:1006A00016F00C94560381E08093880010E00E94BD
:1006B000240662FA16F00C94600381E080938800AF
:1006C00084E190E00E940C050E94130662FA16F085
:1006D0000C946D0381E08093880019E80E94240641
:1006E00062FA16F00C94770381E0809388000E94F0
:1006F0004106A0E9B0E01C9362FA16F00C94830363
:1007000081E0809388000E944106AFE8B0E01C932E
:1007100062FA16F00C948F0381E0809388000E94A7
:100720004106A7E8B0E01C9362FA16F00C949B0314
:1007300081E0809388000E944106A2E9B0E01C930A
:1007400062FA16F00C94A70381E0809388000E945F
:100750004106A1E9B0E01C9362FA16F00C94B303D1
:1007600081E0809388000E944106A7E8B0E01C93D6
:1007700062FA16F00C94BF0381E0809388000E9417
:100780001E06EAE7F3E10E94A004EFE8F0E0A0E52E
:10079000B3E00E9420070E949804EEE8F3E10E9473
:1007A000A004EFE8F0E0A0E5B3E00E94C8060E94D4
:1007B00098040E94A704E2E9F3E10E94A004E1E9A1
:1007C000F0E0A0E5B3E00E9420070E949804EEE864
:1007D000F3E10E94A004E1E9F0E0A0E5B3E00E94AB
:1007E000C8060E9498040E94A704E6ECF1E10E946A
:1007F000D408EFE8F0E0D190E080FF2400270E94C9
:10080000B2070E94DF07EDE0F0E0A3E9B0E00E944C
:100810005107EAECF1E10E94D408E3E9F0E00E941C
:100820007E070E943808EDE0F0E0A3E9B0E00E9406
:100830005107EEECF1E10E94D408E3E9F0E00E94F8
:100840007E070E947708EDE0F0E0A3E9B0E00E94A7
:100850005107E6ECF1E10E94D408E1E9F0E0D19023
:10086000E080FF2400270E94B2070E94DF07EDE02E
:10087000F0E0A7E9B0E00E945107E2EDF1E10E944B
:10088000D408E7E9F0E00E947E070E943808EDE016
:10089000F0E0A7E9B0E00E945107E6EAF3E10E9428
:1008A000A004A0E5B3E0AF93BF93E3E9F0E00E94BA
:1008B0007E070E941B0511E001E0BF91AF910E94ED
:1008C0007206E0E5F3E0A0E5B3E00E944C070E9469
:1008D00098040E94A704E6EBF3E10E94A004A0E5BF
:1008E000B3E0AF93BF93E7E9F0E00E947E070E9478
:1008F0001B0511E001E0BF91AF910E947206E0E597
:10090000F3E0A0E5B3E00E944C070E9498040E9427
:10091000A704E6ECF3E10E94A0040E94A704E6ED20
:10092000F1E10E94A0040E94A7040895F894FFCF6B
:10093000A0E5B3E08D91882311F00CD0FBCF089592
:100940000E946106802D11F005D0FACF08958DE048
:1009500001D08AE05D9BFECF8CB90895A0E5B3E09D
:100960008D91882311F03BD0FBCF08950E94610642
:10097000802D11F034D0FACF089582E03ED01CD003
:1009800012C081E03AD018D080E837C08FE721301C
:1009900039F08FEB223021F08FE8233009F08FEC13
:1009A000810F0C94FD0480E828D0089588EE93E030
:1009B00033D03197D9F7089583E099272DC08AEF76
:1009C00090E00E940C058FEF8ABBBA9ABB9A88E32D
:1009D00014D013D08EE011D086E00FD00895C39AC2
:1009E0008BBBC29AEF93FF93E4ECF0E00E9400050A
:1009F000FF91EF91C2980DD00895C398F1CF08955B
:100A00003197F1F70895689462F80895E89462F8D0
:100A1000089581E090E000C0EF93FF93EE27E82B6C
:100A2000E92B31F0E0EDF7E03197F1F70197D1F7DD
:100A3000FF91EF9108958DE207FD8D938F2D881F13
:100A4000802F881F8F57082F6894F7F8802F87FF13
:100A500015C080958395082F80E38D938EE28D934A
:100A6000802F815228F080E38D9399279C930895DD
:100A700044270A95802F09F196D01FC0805230F08C
:100A80009EE49D9381E48D939D93EFCF4427DF9265
:100A9000EF92FF920F938FE1801B11F0082F83D00C
:100AA00089D09EE29D930F91FF90EF90DF904427B5
:100AB0000395003209F4D7CF2BD03F93E6E4FBE057
:100AC00038E12F2D1E2D0D2DFF24EE24DD2444278B
:100AD000000F111F221FA8F42F923F920E9461065F
:100AE000102C0E946106202C0E946106302C0E946E
:100AF00061063197410DD21CE31CF01C3F902F90F2
:100B000001C0339631963A9519F73F9107D0AFCF90
:100B1000DD0CEE1CFF1C0A95D9F70895002719E09B
:100B200058D08F93802B11F0039501C08F911A95A7
:100B3000B9F7802F882309F496CF8F91805D8D932C
:100B40000A95D9F792CF0065CD1D80B2E60E4059C7
:100B50007307A0ACB90350D6DC01286BEE009435C6
:100B60007700CA9A3B0065CD1D00B2E60E005973AE
:100B70000700ACB90300D6DC01006BEE000035774E
:100B800000009A3B0000CD1D0000E60E0000730738
:100B90000000B9030000DC010000EE000000770057
:100BA00000003B000000F694E794D79447950A951F
:100BB000D1F7089500270DD08F9303958F2D8E299F
:100BC0008D29842BC1F78F91805D8D930A95D9F77C
:100BD0004CCF1F930F93002710E2440FDD1CEE1C37
:100BE000FF1C001F802F9AE0890B10F0082F4395FF
:100BF0001A9599F7802F0F911F910895A198A098A9
:100C0000A99AA89A0895689446BF8F939F938827BE
:100C10009927019621F046B747FFFBCFE8949F91B3
:100C20008F9162F8089544EAEEDF41B1487F483081
:100C300019F0403109F0689462F8089544E946BF1C
:100C400046B744FDFDCF089513B944E8DCDF8F9328
:100C50009F9388279927019669F041B1487F483FC3
:100C6000D1F3E894483139F0483229F0403419F092
:100C7000403509F068949F918F9162F8089544E897
:100C800001C044ECC0DF13B141B1487F483FE1F3FC
:100C9000089501911191219130810895481A590ABE
:100CA0000895481A8827580A089599275A924A920F
:100CB000480E591E08950E9461060D920020D9F732
:100CC0000895C89531960020089599278D919395A0
:100CD0008823E1F7939511968C9311978E919A95AD
:100CE000D1F70895EA2FFB2F00244C918D910394A6
:100CF0008E32E1F711248D9113948823E1F71A9431
:100D0000101640F41197202F2119239580E38D931D
:100D10002A95E9F7113039F59927AE2FBF2FA00D8D
:100D2000B91FA00FB91F8C919C93853308F421C083
:100D300031E08E918E32E9F38D3241F0830F8A33A8
:100D400019F480E331E001C033278C93AE1789F7A3
:100D5000332341F0AE2FBF2FB8DF81E34D3209F4CA
:100D60003196808308958827E00DF81FE00FF81F63
:100D700080830895000F111F221F331F08950095CF
:100D80001095209530950F5F1F4F2F4F3F4F0895BF
:100D9000019110810FC00E9449060EC00E944906B1
:100DA00010C00191108117FF05C03FEF2FEF04C065
:100DB000008111272227332737FF03C0E0DF8DE2B0
:100DC0008D93CF92DF92EF92AA24BB24CC24DD2412
:100DD000EE2440E2EAE0FF2755E093E38081890FAB
:100DE00087FD9F7083FD907F891B81935A95A9F79A
:100DF000C1DFAA1CBB1CCC1CDD1CEE1C4A9551F7A4
:100E0000E894EFE0FF2782910CD0EB30E0F71EF082
:100E100068948A2D0AD088278D93EF90DF90CF9029
:100E20000895982F829501D0892F8F70805D26F0CC
:100E3000803309F4089568948D93089541E003C0C8
:100E400042E001C044E0E40F8827F81F8291982F08
:100E5000829506D0892F04D04A95C1F70C94490792
:100E60008F708A3008F0895F805D8D93089542E02D
:100E700001C041E0E40F8827F81F829138E098E133
:100E8000880F991F9D933A95D1F74A95B1F70C9425
:100E9000490788278D93089581918D938823E1F7E1
:100EA000089594E081918D939A95E1F70895B7FEA6
:100EB000089590E8B91611F4D0FE08959FEFD91A5D
:100EC000E90AF90A09F4039508950F928F939F9305
:100ED000D216E306F4060FB680E890E8802795273F
:100EE0000FBE890739F00FB6892B87FD02C081E05C
:100EF00008260FBE9F918F910F900895D190E19099
:100F0000F19001910895219131914191519108956C
:100F1000502F2D2D3E2D4F2D612F0895D094E0940C
:100F2000F09491E0D90E9927E91EF91E10950895C5
:100F3000652F90E8440F551F5927990F4795607802
:100F4000102F90E8FF0C001F0927990FF7941078D5
:100F500000380895FF0C90E89027110F9795F794AB
:100F6000092F08951127BD2CDE2CEF2CF02E0EE159
:100F7000FF2039F4FE2CED2CDB2CBB240850C2F7EB
:100F800052C032F00A95BB0CDD1CEE1CFF1CF9CFE1
:100F90008EDFE0CF2DEC3CEC4CEC5DE366270FC020
:100FA000ADDFB6DFDD24EE2490E8F92E0FE307C0B5
:100FB000AADF05C02227332740E251E466275523E4
:100FC00051F1002381F1B4DF71F116270058505818
:100FD0000894050B18F407FD03C025C007FD23C0C6
:100FE000469537952795F694E794D79425D0FF201A
:100FF0002AF0DD0CEE1CFF1C015073F09D2D969520
:1010000048F0DD203AF4EE202AF491E0D90E992739
:10101000E91EF91E9FCF07C09FE7092FF92A9FEF0E
:10102000D92EE92E0895DD24EE24FF240027112770
:1010300008950FE79FEFF2CF9F929924AA24BB2433
:1010400088E1D216E306F40628F0D21AE30AF40A7D
:10105000089401C08894991CAA1CBB1CDD0CEE1CD2
:10106000FF1C8A9571F7D92CEA2CFB2C9F900895D0
:101070005FDFD9F05038C9F016270058952F9058E7
:101080000894091F12F418F40EC008F00EC00FD017
:10109000FF202AF0BB0CDD1CEE1CFF1C02C00395D8
:1010A00013F005DF57CF0C940C080C9413089F9293
:1010B000FF92EF928D2DFF24EE24DD24BB2493E0DC
:1010C000849F1001829FB00CD11CE21CF31C839FF3
:1010D000D00CE11C2224F21C9A9531F0BD2CDE2CA0
:1010E000EF2CFF248F91ECCF9F9008950CDF20DF31
:1010F000503829F090E869270CC00AF045D02ACF73
:101100005FE322273327442701C0FDDE11DF50387B
:10111000B1F3003899F3902F951B8BF312F434D070
:10112000FACF983118F0222733274427983028F037
:10113000232F342F44279850F9CF992329F046952F
:10114000379527959A95D9F7912F962742F014D085
:10115000B0F6F794E794D7940F5F8BF65DCF10D07D
:1011600051F008F4DBDEFF2052F2DD0CEE1CFF1C18
:101170000150CBF751CF57CFD20EE31EF41E089586
:10118000D21AE30AF40A0895DF92EF92FF920F93C6
:101190001F93D22EE32EF42E052F162F6F915F9101
:1011A0004F913F912F9108950E946106202D0E943A
:1011B0006106302D0E946106402D0E946106502D6F
:1011C0000895000020C100FF7F4700002F4300006A
:1011D00034420000C84200002A2A2A2A2A2A2A2A3F
:1011E0002A2A204967696E69746F6E20736571756C
:1011F000656E6365207374617274202A2A2A2A2A14
:101200002A2A2A2A2A00487967726F546865726D03
:10121000202056312E3000004D61726B75732046D0
:10122000756C646520273230000052656164536537
:101230007269616C4E756D62657200005265616421
:10124000537461747573466C616773200000536555
:101250007269616C3A20000054656D7020205B005B
:10126000435D3A2030302E30000072656C2E462EE1
:10127000205B255D3A2030302E3000004C756566CD
:101280007465722045494E002A2A20456E746572A5
:10129000204D61696E4C6F6F70202A2A0000534800
:1012A0005438354D6561737572656D656E742D00CA
:1012B00049324320436F6D6D204661696C757265DC
:1012C00000002B2B456E746572205368745F726545
:1012D00061645F73657269616C5F6E756D62657282
:1012E000000053657269616C204E756D62657220F5
:1012F0003A2000002D2D4C656176696E6720536899
:10130000745F726561645F73657269616C5F6E754D
:101310006D62657200002B2B456E746572205368F8
:10132000745F726561645F7374617475735F627911
:101330007465730053746174757320466C616773D0
:10134000203A20002D2D456E746572205368745F1D
:10135000726561645F7374617475735F62797465DB
:1013600073002B2B456E746572205368745F6D6536
:1013700061737572656D656E7400524157205465D6
:101380006D7065726174757265203A200000203DB1
:1013900020005241572048756D6964697479202096
:1013A00020203A20000054656D706572617475727A
:1013B00065203A20000048756D69646974792020C1
:1013C00020203A2000002D2D456E74657220536850
:0E13D000745F6D6561737572656D656E740096
:00000001FF
